:107800000C942A3C0C94473C0C94473C0C94473C09
:107810000C94473C0C94473C0C94473C0C94473CDC
:107820000C94473C0C94473C0C94473C0C94473CCC
:107830000C94473C0C94473C0C94473C0C94473CBC
:107840000C94473C0C94473C0C94473C0C94473CAC
:107850000C94473C11241FBECFE5D8E0DEBFCDBF5E
:1078600010E0A0E6B0E0EEEFFEE702C005900D925A
:10787000A036B107D9F711E0A0E6B0E001C01D9233
:10788000A43AB107E1F70E94363F0C947D3F0C9477
:10789000003C0F92AF93BF93CF93DF93EF93FF938F
:1078A000FC01EA01DB01C895099231961197D9F7DD
:1078B000FF91EF91DF91CF91BF91AF910F9008951C
:1078C0000F921F920F931F93AF93BF93CF93DF93AA
:1078D000EF93FF93FC01EA01DB0110E80990199096
:1078E00001E04CD03296129711F01250B9F7FC011A
:1078F00003E044D005E042D000E810E0800F911F83
:10790000109759F7FF91EF91DF91CF91BF91AF9110
:107910001F910F911F900F9008950F931F93EF9356
:10792000FF93FC0103E02AD000E810E0E00FF11F14
:10793000E617F707B9F7FF91EF911F910F9108959F
:107940000F930F9222D0082E09E018D00F900F91BC
:1079500008950F930F92EF93FF9317D0FC0160935C
:107960005700C895802DFF91EF910F900F910895CA
:107970000F930BD001E102D00F910895E199FECF52
:1079800000935700E895FFFF00000091570000FDAD
:10799000FCCF089588E089B98AB188618AB90895D1
:1079A0008AB1877E8AB908958CB95E9BFECF5E9AB4
:1079B00008958CB108958BB180780895AC0120E0D2
:1079C00030E009C05F9BFECF8CB1FA01E20FF31FDC
:1079D00080832F5F3F4F26173707A0F381E008957C
:1079E000FC0120E030E008C080818CB95E9BFECFB6
:1079F00031965E9A2F5F3F4F26173707A8F381E035
:107A00000895813879F0823818F4803839F408C044
:107A1000823851F0883911F483E0089580E00895A8
:107A200082E0089581E0089582E108956091A000C8
:107A30007091A1004091A2015091A30120E030E09B
:107A400010C0C901840F951F9FBB8EBBF901EE5575
:107A5000FF4F80818DBBE29AE19AE199FECF2F5FC3
:107A60003F4F2617370768F3460F571F5093A30160
:107A70004093A20108956091A0007091A1004091EF
:107A8000A2015091A30120E030E00DC0C901840F94
:107A9000951F9FBB8EBBE09A8DB3F901EE55FF4F4A
:107AA00080832F5F3F4F2617370780F3460F571FFE
:107AB0005093A3014093A201089540E050E00BC011
:107AC00020E030E000002F5F3F4F67E0203D3607A9
:107AD000C9F74F5F5F4F4817590790F308956091BA
:107AE000A0007091A1008091A2019091A30142EAAF
:107AF00050E0880F991F0E94493C0895CF93DF936F
:107B0000C0E0D0E011C0AE014E555F4F8091A201A0
:107B10009091A301880F991F60E870E08C0F9D1F62
:107B20000E94603CC058DF4F8091A0009091A1005E
:107B3000C817D90740F30E94B83CDF91CF91089550
:107B40000E94DB3C8823E1F30E94D93C803211F48F
:107B500081E0089585E10E94D43C80E00895DF92A1
:107B6000EF92FF920F931F93CF93DF9369E081E031
:107B700090E00E94A93C84FF03C08F7E0E94A03C3D
:107B8000DD240E94DB3C8823E1F30E94D93C82354E
:107B9000C0F4803508F078C0813409F443C08234E1
:107BA00048F4813321F1803409F452C1803309F063
:107BB0004BC16AC0823409F458C0853409F044C10D
:107BC00057C0863509F40DC1873538F4823509F47C
:107BD00061C0853509F038C16CC0843709F4A6C08E
:107BE000853709F4EEC0843609F02EC17AC00E94B0
:107BF000A03D882331F284E10E94D43C81E40E94BC
:107C0000D43C86E50E94D43C82E50E94D43C80E2CC
:107C10000E94D43C83E50E94D43C84E50E94D43C7D
:107C20008BE40EC161E070E080E690E00E94DE3CF3
:107C30000E94A03D882309F4A4CF84E10E94D43C93
:107C400080916000813869F0823818F4803839F406
:107C5000C6C0823841F0883911F483E0F1C080E079
:107C6000EFC081E0EDC082E1EBC064E170E008C0EC
:107C700061E070E080E690E00E94DE3C64E070E04D
:107C800080E690E00E94DE3C0E94A03D882309F43B
:107C900078CF0DC00E94A03D882309F472CF60E028
:107CA00070E880E090E00E948D3C0E94B83C84E146
:107CB000C7C062E070E080E690E00E94DE3C0E9477
:107CC000A03D882309F45DCFF0906100EE248091FF
:107CD00060009701280F311D3093A3012093A2016A
:107CE000E6CF63E070E080E690E00E94DE3CD09159
:107CF0006000C0E080916100BE01680F711D70934B
:107D0000A1006093A00082EA90E00E94DE3C0E9405
:107D1000A03D882309F435CF80916200863419F4A0
:107D20000E947E3DC4CF0E94163DC1CF63E070E04B
:107D300080E690E00E94DE3C1091600000E08091BF
:107D400061009801280F311D3093A1002093A000FD
:107D50000E94A03D882309F414CF809162008634EC
:107D600059F04091A0005091A1006091A201709142
:107D7000A30120E030E010C00E946F3D16C0C90191
:107D8000860F971F9FBB8EBBE09A8DB3F901EE550E
:107D9000FF4F80832F5F3F4F2417350780F3460F37
:107DA000571F5093A3014093A20184E10E94D43C49
:107DB0006091A0007091A10082EA90E00E94F03CE6
:107DC00041C00E94A03D882309F4DBCE84E10E94DB
:107DD000D43C8EE10E94D43C85E90E94D43C82E0F0
:107DE0002FC064E070E080E690E00E94DE3C0E94DC
:107DF000A03D882309F4C5CE84E10E94D43C809143
:107E00006000803531F480916100882359F4DD24CD
:107E100012C0883581F480916100883041F453E0CC
:107E2000D52E09C0883039F442E0D42E04C088230E
:107E300011F4DD24D39469E08D2D90E00E94A93CDB
:107E40000E94D43C80E101C085E10E94D43C99CEDF
:107E5000DF91CF911F910F91FF90EF90DF900895E8
:107E60000E94D03CE0E0F0E0099508951F93F8945B
:107E7000E199FECF8EEF93E09FBB8EBBE09A8DB36E
:107E8000843B99F4E199FECF8FEF93E09FBB8EBBCB
:107E9000E09A8DB3833C49F4E199FECF8DEF93E0F6
:107EA0009FBB8EBBE09A8DB381BF0E94CA3C0E94EB
:107EB000D93C1EE119C00000019647E0803D9407BF
:107EC000D1F72F5F3F4F2436310519F080E090E065
:107ED000F2CF0E94DB3C882319F00E94AF3D07C01F
:107EE000115018BB112319F020E030E0EFCF0E94B1
:0E7EF000303F80E090E01F910895F894FFCF9E
:040000030000780081
:00000001FF
